:020000040000FA
:1000000000001B0AF80C670106020F0F0F0E000814
:100010000C02E201820814081208110824082208C0
:100020002108440842084108840881080107160A8B
:100030000106180A00086400860C0200FF0C060086
:10004000F00C07006A000A02280043072C0A020984
:1000500043062B0AAA02620AE8004307540A0B0C63
:100060002C00070C270108092B00070EA7018B03A2
:100070000F0E460143073D0A410AFF0CEC0103063F
:10008000310A4307520AF60CCC0103064A0A300C27
:10009000CC014F0A43074E0A2A0C4F0A230C2D00AD
:1000A000AA02530A6A00620AE80043075C0A0209CE
:1000B00043075B0AAA02620A02094307610A6A004F
:1000C000620AEA002D024306760A16096704080C44
:1000D00028002D03160903076F0A6705700A6704D5
:1000E000E8004307690A160967056D00040001026C
:1000F0002800E9077E0AE8067E0A800A2900760AB7
:040100002900230AA5
:021FFE00DA0FF8
:00000001FF
